:100000000C9484000C94AC000C94AC000C94240A66
:100010000C94240A0C94240A0C94AC000C94410710
:100020000C94AC000C94AC000C94AC000C94300814
:100030000C94AC000C94AC000C94AC000C94AC0090
:100040000C948F0C0C94AC000C94DB0F0C940D10E2
:100050000C94AC000C94AC000C94AC000C94AC0070
:100060000C94620B0C94AC0000000008000201002C
:100070000003040700000000000000000102040863
:100080001020408001020408102001020408102002
:10009000040404040404040402020202020203032E
:1000A00003030303000000002300260029000000D2
:1000B0000000250028002B0000000000240027007D
:1000C0002A004E414E494E495459494E46CDCCCC5A
:1000D0003D0AD7233C17B7D13877CC2B329595E61C
:1000E000241FB14F0A000020410000C84200401CFC
:1000F0004620BCBE4CCA1B0E5AAEC59D740062069B
:100100000F07350B3D10130711241FBECFEFD8E0AA
:10011000DEBFCDBF11E0A0E0B1E0EAECF0E302C049
:1001200005900D92AC39B107D9F725E0ACE9B1E003
:1001300001C01D92A53CB207E1F710E0C6E0D1E096
:1001400004C02297FE010E94E615CE3FD107C9F7F1
:100150000E94E7120C9458180C9400001816190607
:1001600014F460E001C061E084E092E00E940608BF
:1001700061E084E092E00E94160860E084E092E092
:100180000C9416081816190614F460E001C061E01A
:1001900080E092E00E94060861E080E092E00E9428
:1001A000160860E080E092E00C9416082F923F92CF
:1001B0004F925F926F927F928F929F92AF92BF9277
:1001C000CF92DF92EF92FF920F931F93CF93DF9323
:1001D000CDB7DEB762970FB6F894DEBF0FBECDBFC6
:1001E00080910A0190910B012C01662457FC6094C8
:1001F000762C209012023090130280910E02909182
:100200000F02281A390A00911002109111028091F0
:100210000C0290910D02081B190B680117FF04C016
:10022000CC24DD24C01AD10A910137FE04C0222754
:1002300033272219330979012C153D050CF4760179
:10024000B701882777FD8095982F298B3A8B0E94DC
:10025000FB134B015C0129893A89B901882777FD95
:100260008095982F0E94FB13A50194010E946013B2
:100270006D837E838F839887B601882777FD80956D
:10028000982F0E94FB13A50194010E9460136987B7
:100290007A878B879C87FA82E982812C912C540182
:1002A000750164012FEF3FEF3C832B83E0910E0239
:1002B000F0910F02FE87ED87809112029091130258
:1002C000E817F90709F4EBC02D813E814F8158856D
:1002D000C701B6010E94F8126B017C0120E030E0FA
:1002E00040E85FE30E94B91487FD27C0121413048D
:1002F0001CF480910B0202C080910A02992787FDAD
:100300009095121413041CF421E030E002C02FEF8A
:100310003FEF4D855E85240F351F30930F022093EC
:100320000E020E94AE0020E030E040E85FE3C7012B
:10033000B6010E94F7126B017C0180910C02909132
:100340000D029E878D878091100290911102ED859C
:10035000FE85E817F907C9F129853A854B855C8543
:10036000C501B4010E94F8124B015C0120E030E0AD
:1003700040E85FE30E94B91487FD27C010161106FC
:100380001CF48091090202C080910802992787FD20
:100390009095101611061CF421E030E002C02FEFFA
:1003A0003FEF4D855E85240F351F30930D0220935E
:1003B0000C020E94C20020E030E040E85FE3C5018B
:1003C000B4010E94F7124B015C01EB81FC81CF016B
:1003D000AA2797FDA095BA2F840D951DA61DB71DC0
:1003E00020910C0130910D01A901662757FD609500
:1003F000762F84179507A607B7076CF040910A017E
:1004000050910B01662757FD6095762F48175907C5
:100410006A077B0714F4DB01CA014090DD015090AC
:10042000DE016090DF017090E001480E591E6A1EE7
:100430007B1EF1E14F16F7E25F06610471049CF048
:10044000C301B20128EE33E040E050E00E94AB155A
:100450006D877E878F87988BCA01B9010E94080D2E
:100460008D859E8501C0C2010E94300D80910A01D8
:1004700090910B0120910C0130910D01821B930B87
:1004800029813A812817390724F441E050E05C8340
:100490004B8389819A8101979A83898307CF209121
:1004A00010023091110280910C0290910D0282177E
:1004B000930709F042CF62960FB6F894DEBF0FBEE5
:1004C000CDBFDF91CF911F910F91FF90EF90DF9003
:1004D000CF90BF90AF909F908F907F906F905F90E4
:1004E0004F903F902F9008954F925F926F927F921E
:1004F0008F929F92AF92BF92CF92DF92EF92FF9234
:10050000CF93DF9300D000D0CDB7DEB7C0901C02F0
:10051000D0901D02E0901E02F0901F022091240254
:10052000309125024091260250912702C701B60161
:100530000E94F7122B013C01809118029091190240
:10054000A0911A02B0911B0289839A83AB83BC836A
:1005500020912002309121024091220250912302E9
:10056000BC01CD010E94F7124B015C01A301920175
:10057000C301B2010E94BD142B013C01A5019401ED
:10058000C501B4010E94BD149B01AC01C301B201BD
:100590000E94F8120E9424152FE632E143E85AE344
:1005A0000E945C1387FD52C020E030E048E455E42F
:1005B000C701B6010E94BD1420E030E044EB53E4D3
:1005C0000E9460130E94C81370931302609312027A
:1005D00020E030E048E455E469817A818B819C8198
:1005E0000E94BD1420E030E044EB53E40E9460130D
:1005F00020E030E040EA50E40E94BD140E94C8139D
:1006000070931102609310020E94D60080911C0228
:1006100090911D02A0911E02B0911F0280932402AE
:1006200090932502A0932602B0932702809118028E
:1006300090911902A0911A02B0911B02809320029E
:1006400090932102A0932202B09323020F900F9067
:100650000F900F90DF91CF91FF90EF90DF90CF90B0
:10066000BF90AF909F908F907F906F905F904F90D2
:1006700008951092240210922502109226021092E0
:10068000270280E090E0A0E7B2E4809320029093FC
:100690002102A0932202B093230210920F02109223
:1006A0000E028AE69AE090930D0280930C02089560
:1006B000CF93DF9300D0CDB7DEB7409124025091A5
:1006C0002502609126027091270240931C025093EC
:1006D0001D0260931E0270931F02409120025091F0
:1006E00021026091220270912302409318025093DC
:1006F000190260931A0270931B02AE014F5F5F4FA5
:1007000063E371E00E944916AE014F5F5F4F63E300
:1007100071E080E090E00E944916009709F44FC014
:10072000FC012081283561F401960E94EA1560934E
:100730001C0270931D0280931E0290931F02E4CF4F
:10074000293561F401960E94EA15609318027093AE
:10075000190280931A0290931B02D6CF2A3561F4B6
:1007600001960E94EA15609314027093150280931B
:10077000160290931702C8CF263491F401960E9476
:10078000EA1520E030E040E752E40E9460136093F5
:1007900028027093290280932A0290932B02B4CFEF
:1007A000213409F0B1CF01960E940C166093DD014F
:1007B0007093DE018093DF019093E001A5CF0E944A
:1007C00074020F900F90DF91CF9108956CE271E069
:1007D00086E295E00E94BE1022E030E040E050E06A
:1007E00068E475E486E295E00E948B1260E286E29E
:1007F00095E00E94C0104091240250912502609122
:1008000026027091270222E030E086E295E00E9405
:100810008B1260E286E295E00E94C01040912002B7
:1008200050912102609122027091230222E030E077
:1008300086E295E00E948B1265E371E086E295E026
:100840000E94BE106091340270E04AE050E086E2FF
:1008500095E00E94801168E371E086E295E00E94D5
:10086000BE106091350270E04AE050E086E295E00B
:100870000E9480116BE371E086E295E00E94BE1059
:1008800060913602709137024AE050E086E295E0CE
:100890000E9480116EE371E086E295E00E94BE1036
:1008A00060913802709139024AE050E086E295E0AA
:1008B0000E94801161E471E086E295E00E94BE1022
:1008C00060913A0270913B024AE050E086E295E086
:1008D0000C948811CF93DF9300D0CDB7DEB7AE0173
:1008E0004F5F5F4F63E371E00E94491689819A81EF
:1008F0000E940C166093DD017093DE018093DF018E
:100900009093E0010F900F90DF91CF910895CF93D6
:10091000DF9300D0CDB7DEB7AE014F5F5F4F63E32B
:1009200071E00E94491689819A810E94EE15BC01EE
:100930008AEE91E00E94E6060F900F90DF91CF9132
:100940000895CF93DF9300D0CDB7DEB7AE014F5FF0
:100950005F4F63E371E00E94491689819A810E948A
:10096000EE15BC0181EE91E00E94BF090F900F903F
:10097000DF91CF910895CF93DF93EC010E94EE15A4
:1009800081309105D1F04C97E9F410921C0210923D
:100990001D0210921E0210921F0280E090E0A0E75C
:1009A000B2E48093180290931902A0931A02B093B4
:1009B0001B02DF91CF910C947402CE01DF91CF9195
:1009C0000C945803DF91CF9108950F931F93CF9309
:1009D000DF930CE212E0C0E0D0E0F80161918F01FA
:1009E000CE010E9495162196C034D105B1F7DF9152
:1009F000CF911F910F9108950F931F93CF93DF9382
:100A000000D0CDB7DEB7AE014F5F5F4F63E371E05B
:100A10000E9449168C01012B49F1AE014F5F5F4FD7
:100A200063E371E080E090E00E9449168C01FC01D4
:100A30008081813439F4C80101960E94EE158093BB
:100A40003402E9CF823439F4C80101960E94EE15D0
:100A500080933502E0CF8434F1F6C80101960E94FC
:100A6000EE159093370280933602D5CF0E94E504AD
:100A70000F900F90DF91CF911F910F9108950F93D9
:100A80001F93CF93DF9300D0CDB7DEB7AE014F5F9A
:100A90005F4F63E371E00E9449168C01012B11F155
:100AA000AE014F5F5F4F63E371E080E090E00E9432
:100AB00049168C01FC018081853549F4C8010196F5
:100AC0000E94EE159093390280933802E7CF843468
:100AD00029F7C80101960E94EE1590933B0280937E
:100AE0003A02DCCF0E94E5040F900F90DF91CF9186
:100AF0001F910F910895CF93DF93EC010E94EE15A3
:100B000083309105D1F054F48130910589F002973A
:100B100019F5CE01DF91CF910C943F0585309105F9
:100B2000B1F084F00A97C1F4DF91CF910C94E60301
:100B3000CE01DF91CF910C94A104CE01DF91CF9132
:100B40000C946A04CE01DF91CF910C948704CE01FE
:100B5000DF91CF910C94FC04DF91CF910895FC01BB
:100B60002081273421F401960E94BB0430C02D342B
:100B700021F401960E947B052AC0203541F564E4EA
:100B800071E086E295E00E94BE10409124025091EF
:100B90002502609126027091270222E030E086E271
:100BA00095E00E948B126AE471E086E295E00E9473
:100BB000BE1040912002509121026091220270915A
:100BC000230222E030E086E295E00E948D126DE47F
:100BD00071E086E295E00C94CB100F931F93CF93B6
:100BE000DF930CE212E0C0E0D0E0CE010E948D164F
:100BF000D8018D938D012196C034D105B1F744E021
:100C000050E060E571E08CE292E00E943B16892B97
:100C1000D9F065E571E086E295E00E94CB1080E4B2
:100C2000ECE2F2E0DF011D928A95E9F785E497E4B2
:100C3000A7E4B3E380932C0290932D02A0932E029D
:100C4000B0932F020E94E50480913402811105C007
:100C500081E080930B028FEF04C08FEF80930B0233
:100C600081E080930A0280913502811105C08FEFE7
:100C70008093090281E004C081E0809309028FEF34
:100C800080930802DF91CF911F910F91089526E084
:100C900040E052EC61E070E086E295E00E94790F5E
:100CA0000E94ED050E9439036091E4017091E50115
:100CB00081EE91E00E94860960E070E081EE91E0B3
:100CC0000C94BF0961E084E092E00E94F60762E0C4
:100CD00080E092E00E94F60763E08CEF91E00E94D2
:100CE000F6078CEF91E00E942A0890E09093FB01B8
:100CF0008093FA018CEF91E00E942D0890E0909390
:100D0000F9018093F80166E084EF91E00E94F60714
:100D100084EF91E00E942A0890E09093F301809381
:100D2000F20184EF91E00E942D0890E09093F10190
:100D30008093F0016AE08AEE91E00E94E40667E0A9
:100D400086EE91E00E94F60786EE91E00E942D0863
:100D500090E09093E5018093E40181EE91E00C94A2
:100D6000EC0886E295E00E94960E892B61F186E2FE
:100D700095E00E94AF0EE0919C018A30C1F481E0C1
:100D80008E0F80939C01FF27E7FDF095E356FE4F01
:100D900010828DE991E00E94AF0580E4EDE9F1E079
:100DA000DF011D928A95E9F710929C010895E034C5
:100DB00054F491E09E0F90939C01FF27E7FDF0957E
:100DC000E356FE4F808308950C94F6070F931F930C
:100DD000CF93DF938C016F3F710519F014F06FEF23
:100DE00070E0EB0161308FEF780714F4C1E0DFEFC2
:100DF000D7FD06C061E0C8010E941608BE0108C008
:100E000060E0C8010E941608662777276C1B7D0BDF
:100E1000C801DF91CF911F910F910C9426088CE6A9
:100E200092E00C9417078CE692E00C94400721E0C6
:100E300030E0FC0131832083EE5FFE4F108211828F
:100E40001282138234961082118212821382349697
:100E50001082319610823196108211821282138292
:100E6000349611821082329610823196108211824D
:100E70001282138234961082118212821382089594
:100E800008951F920F920FB60F9211240F931F9384
:100E90002F933F934F935F936F937F938F939F9382
:100EA000AF93BF93CF93EF93FF9382E00E946D0EB9
:100EB000C82F20918D0330918E032F5F3F4F3093C9
:100EC0008E0320938D038091F303843618F085E020
:100ED0008093880390918803933079F018F49230CE
:100EE00039F070C0943011F1953009F44AC06AC0ED
:100EF000C11168C01092F30329C0C13009F062C06B
:100F0000E091F30381E08E0F8093F303F0E0809192
:100F10008D0390918E03E957FC4F808710928E03CA
:100F200010928D0384E0809388034CC0C11114C0DB
:100F3000E091F30381E08E0F8093F303F0E0809162
:100F40008D0390918E03E957FC4F808710928E039A
:100F500010928D0383E0E7CF80918D0390918E03F3
:100F60008536910578F185E0809388030E94D90C3D
:100F70006093890370938A0380938B0390938C030F
:100F800021C00E94D90C0091890310918A032091FD
:100F90008B0330918C03601B710B820B930B693CAC
:100FA00071058105910540F01092F30310928E03B4
:100FB00010928D0382E0B7CFC11104C010928E034E
:100FC00010928D03FF91EF91CF91BF91AF919F91BF
:100FD0008F917F916F915F914F913F912F911F91D1
:100FE0000F910F900FBE0F901F901895DC01E62F08
:100FF000F0E0EE0FFF1FE25FFE4F80818C93818156
:1010000011968C93119712966C9308951F93CF931A
:10101000DF93EC01162F61E088810E94FE0D612FA5
:101020008881DF91CF911F910C94370E1F93CF933E
:10103000DF93EC01162F61E089810E94FE0D612F84
:101040008981DF91CF911F910C94370EFC01808133
:101050000C94760DFC0180810895FC018181089536
:101060001F920F920FB60F9211242F933F934F931D
:101070005F936F937F938F939F93AF93BF93EF9300
:10108000FF938091F50387FF05C0109285001092B1
:1010900084001AC02091F503332727FD30958091F5
:1010A000F40390E0281739077CF48091F503992721
:1010B00087FD9095FC01EE0FFF1FE80FF91FEA5026
:1010C000FC4F808187FD15C08091F5038F5F809371
:1010D000F5032091F503332727FD30958091F40324
:1010E00090E028173907BCF48091F5038C305CF14F
:1010F00012C08091F503992787FD9095FC01EE0FB2
:10110000FF1FE80FF91FEA50FC4F808160E08F77E6
:101110000E94370ED9CF809184009091850004966B
:1011200080349C4918F480E49CE905C080918400D7
:1011300090918500049690938900809388008FEFAA
:101140008093F50338C02091840030918500809110
:10115000F503992787FD9095FC01EE0FFF1FE80F1F
:10116000F91FEA50FC4F81819281820F931F909367
:101170008900809388008091F503992787FD9095D9
:10118000FC01EE0FFF1FE80FF91FEA50FC4F8081B2
:1011900087FF11C08091F503992787FD9095FC0189
:1011A000EE0FFF1FE80FF91FEA50FC4F808161E04E
:1011B0008F770E94370EFF91EF91BF91AF919F9172
:1011C0008F917F916F915F914F913F912F910F90F0
:1011D0000FBE0F901F9018952091F4032C30A0F4AF
:1011E00031E0320F3093F403FC012083822F90E032
:1011F000FC01EE0FFF1FE80FF91FEA50FC4F88EBD0
:101200009BE09283818308952FEFFC012083089552
:10121000DF92EF92FF920F931F93CF93DF93EC0136
:10122000D62E7A01890188818C3008F066C061E091
:101230008D2D0E94FE0D8881A82FB0E0FD01EE0FDC
:10124000FF1FEA0FFB1FEA50FC4F2D2D2F779081D7
:101250009078922B908360E272E06E197F0977FF9D
:1012600002C06D5F7F4F759567957595679569832A
:1012700040E659E0401B510B57FF02C04D5F5F4FE6
:1012800055954795559547954A836CE00E947D1585
:101290009CE0899FB001112420E030E0A901460FB5
:1012A000571FFA01EE0FFF1FE40FF51FEA50FC4F26
:1012B000908197FD16C02F5F3F4F2C30310571F79D
:1012C00081110FC01092800082E080938100109203
:1012D000850010928400B19A80916F0082608093A3
:1012E0006F00888190E0FC01EE0FFF1FE80FF91FEF
:1012F000EA50FC4F8081806880838881DF91CF91A4
:101300001F910F91FF90EF90DF90089520E639E054
:1013100040E252E00C940809FC0180818C3070F5A9
:10132000918128E830E0291B310997FD3395220F80
:10133000331F220F331F621773077CF0928128E559
:1013400032E0291B310997FD3395220F331F220FFD
:10135000331F621773070CF49B0122503109220FCF
:10136000331F4FB7F89490E0FC01EE0FFF1FE80F1A
:10137000F91FEA50FC4F328321834FBF08954F92EB
:101380005F926F927F92AF92BF92CF92DF92EF9275
:10139000FF920F931F93CF93DF93EC01603282E0B3
:1013A00078070CF040C077FD06C0653B71052CF056
:1013B00064EB70E002C060E070E0898128E830E012
:1013C000281B310987FD3395220F331F220F331F4E
:1013D0005901CC24B7FCC094DC2C882777FD80957C
:1013E000982F2A8148E552E0421B510927FD539569
:1013F000440F551F440F551F2A01662457FC609463
:10140000762C7F926F925F924F9214EBE12EF12C2B
:1014100000E010E020E030E0A9010E949F120F9050
:101420000F900F900F90CE01DF91CF911F910F91F0
:10143000FF90EF90DF90CF90BF90AF907F906F9034
:101440005F904F900C948C091F920F920FB60F92E1
:1014500011242F933F934F935F936F937F938F93B9
:101460009F93AF93BF93EF93FF93E0915C04F09150
:101470005D04309709F451C0868DA685B7859585A2
:1014800081FF04C08C91892329F447C08C91892362
:1014900009F043C0A389B4899C91858980958923EB
:1014A0008C93868997890197F1F7208D318DA685D8
:1014B000B785758558E040E0C9010197F1F7842FA1
:1014C00090E095958795482F6C91672309F04068C7
:1014D000515091F7868D81FD409580911B0490E0DD
:1014E00001968F73992720911A04281749F0A0912B
:1014F0001B04B0E0A45EBB4F4C9380931B0403C05D
:10150000868D8160868F828D938D0197F1F7A389F7
:10151000B4898C919589892B8C93FF91EF91BF9120
:10152000AF919F918F917F916F915F914F913F917B
:101530002F910F900FBE0F901F90189580918D04E2
:1015400090E020918E04821B9109089520918E04D1
:1015500080918D04281750F4E22FF0E0E157FB4F03
:10156000808190E02F5F20938E0408958FEF9FEF8E
:101570000895E0918E0480918D04E81730F4F0E036
:10158000E157FB4F808190E008958FEF9FEF089522
:101590000895CF92DF92EF92FF920F931F93CF9314
:1015A000DF937C01CB018A0120916A04222389F018
:1015B000EB016B01C40ED51ECC15DD0569F06991F8
:1015C000D701ED91FC910190F081E02DC7010995C3
:1015D000F3CF642F0E94390BC801DF91CF911F9187
:1015E0000F91FF90EF90DF90CF900895CF93DF930E
:1015F0001F92CDB7DEB7698320916A042223D1F010
:1016000020916B04203240F021E030E0FC01338374
:10161000228380E090E015C080916C04E82FF0E018
:10162000E359FB4F998190838F5F80936C04809383
:101630006B0405C061E0CE0101960E94390B81E088
:1016400090E00F90DF91CF910895FC0113821282F8
:1016500048EE53E060E070E044835583668377830F
:101660008EE691E09183808308958EE594E00C945A
:10167000250B613298F420911C05243089F4609385
:10168000D104FC0183ED94E0DC012A2F281B2617EE
:1016900018F421912D93F9CF80E0089581E0089509
:1016A00082E0089585ED8093BC008091BC0084FDAC
:1016B000FCCF10921C05089585EC8093BC0010921D
:1016C0001C0508951F920F920FB60F9211242F93AD
:1016D0003F934F935F936F937F938F939F93AF93BA
:1016E000BF93EF93FF938091B900887F803609F410
:1016F0009EC078F5883209F45DC090F4803109F419
:1017000056C038F4882309F4F5C0883009F44FC076
:10171000F5C0883109F44EC0803209F45FC0EEC0D4
:10172000803409F46AC058F4803309F457C0883310
:1017300009F0E4C08093AF040E945C0BDFC08035E9
:1017400009F44FC0883509F45DC0883409F0D6C06B
:10175000D3C0883909F4C4C0A8F4883709F467C035
:1017600038F4883609F463C0803709F460C0C6C015
:10177000883809F4B5C0803909F45FC0803809F0B1
:10178000BDC05BC0803B09F483C038F4803A09F4E3
:1017900066C0883A09F47CC0B1C0803C09F4A4C09A
:1017A000883C09F4A1C0883B09F487C0A7C0809198
:1017B0001B0510C09091F4048091F304981770F504
:1017C000E091F40481E08E0F8093F404F0E0EB509C
:1017D000FB4F80818093BB0085EC83C08093AF0476
:1017E0008BC0E091F40481E08E0F8093F40480912B
:1017F000BB00F0E0EB50FB4F80839091F4048091AC
:10180000F3046BC0E091F40481E08E0F8093F40444
:101810008091BB00F0E0EB50FB4F808380911A0574
:1018200081116AC081E08093190584EA5EC083E07B
:1018300080931C051092B004CFCF8091B004803209
:1018400008F04EC0E091B00481E08E0F8093B004A8
:101850008091BB00F0E0EF54FB4F8083BDCF0E942E
:101860005C0B8091B004803230F4E091B004F0E081
:10187000EF54FB4F10826091B00470E0E0911505C9
:10188000F091160581EB94E009951092B00436C0F2
:1018900084E080931C051092D2041092D104E09150
:1018A0001705F091180509958091D104811105C0A3
:1018B00081E08093D1041092D304E091D20481E0BE
:1018C0008E0F8093D204F0E0ED52FB4F8081809325
:1018D000BB009091D2048091D104981708F47CCF7A
:1018E00085E88093BC000AC085EC8093BC00109210
:1018F0001C0504C01092AF040E94520BFF91EF919F
:10190000BF91AF919F918F917F916F915F914F9117
:101910003F912F910F900FBE0F901F9018951F921F
:101920000F920FB60F9211242F933F938F939F9393
:10193000AF93BF9380911E0590911F05A091200544
:10194000B091210530911D0523E0230F2D3720F4A0
:101950000196A11DB11D05C026E8230F0296A11D09
:10196000B11D20931D0580931E0590931F05A09324
:101970002005B09321058091220590912305A09127
:101980002405B09125050196A11DB11D8093220566
:1019900090932305A0932405B0932505BF91AF91A3
:1019A0009F918F913F912F910F900FBE0F901F909D
:1019B00018952FB7F89460911E0570911F058091BE
:1019C0002005909121052FBF08953FB7F89480918D
:1019D000220590912305A0912405B091250526B5F7
:1019E000A89B05C02F3F19F00196A11DB11D3FBF57
:1019F0006627782F892F9A2F620F711D811D911DE7
:101A000042E0660F771F881F991F4A95D1F7089506
:101A1000CF92DF92EF92FF92CF93DF936B017C0125
:101A20000E94E50CEB01C114D104E104F10489F03A
:101A30000E94F6120E94E50C6C1B7D0B683E734001
:101A400090F381E0C81AD108E108F108C851DC4FD1
:101A5000EACFDF91CF91FF90EF90DF90CF90089584
:101A60008230910538F0880F991F880F991F0597CC
:101A70000197F1F70895789484B5826084BD84B5A8
:101A8000816084BD85B5826085BD85B5816085BD79
:101A9000EEE6F0E0808181608083E1E8F0E0108292
:101AA000808182608083808181608083E0E8F0E0D3
:101AB000808181608083E1EBF0E0808184608083BD
:101AC000E0EBF0E0808181608083EAE7F0E08081F4
:101AD0008460808380818260808380818160808354
:101AE0008081806880831092C10008951F93CF93F6
:101AF000DF93182FEB0161E00E94FE0D209711F497
:101B000060E004C0CF3FD10539F461E0812FDF915F
:101B1000CF911F910C94370EE12FF0E0E859FF4F61
:101B2000E491E330F9F048F4E130B9F0E230A1F5A6
:101B300084B5806284BDC8BD34C0E730E9F0E830C8
:101B400019F1E43049F58091800080628093800033
:101B5000D0938B00C0938A0024C084B5806884BD74
:101B6000C7BD1FC080918000806880938000D093A3
:101B70008900C093880015C08091B0008068809370
:101B8000B000C093B3000DC08091B000806280931C
:101B9000B000C093B40005C0C038D1050CF0B5CF7B
:101BA000AFCFDF91CF911F910895833081F028F45A
:101BB000813099F08230A1F008958730A9F0883003
:101BC000B9F08430D1F4809180008F7D03C0809182
:101BD00080008F7780938000089584B58F7702C04E
:101BE00084B58F7D84BD08958091B0008F7703C048
:101BF0008091B0008F7D8093B0000895CF93DF93E4
:101C000090E0FC01E458FF4F2491FC01E057FF4FA6
:101C10008491882349F190E0880F991FFC01E854D2
:101C2000FF4FA591B49182559F4FFC01C591D4916E
:101C30009FB7611108C0F8948C91209582238C93F2
:101C4000888182230AC0623051F4F8948C91322F3B
:101C5000309583238C938881822B888304C0F894E9
:101C60008C91822B8C939FBFDF91CF9108950F931E
:101C70001F93CF93DF931F92CDB7DEB7282F30E0AD
:101C8000F901E859FF4F8491F901E458FF4F14918D
:101C9000F901E057FF4F04910023C9F0882321F098
:101CA00069830E94D50D6981E02FF0E0EE0FFF1FE0
:101CB000E255FF4FA591B4919FB7F8948C916111B3
:101CC00003C01095812301C0812B8C939FBF0F907F
:101CD000DF91CF911F910F910895CF93DF93282F1C
:101CE00030E0F901E859FF4F8491F901E458FF4FC2
:101CF000D491F901E057FF4FC491CC2391F08111A9
:101D00000E94D50DEC2FF0E0EE0FFF1FEC55FF4FBA
:101D1000A591B4912C912D2381E090E021F480E0F5
:101D200002C080E090E0DF91CF910895FC01818DA9
:101D3000228D90E0805C9F4F821B91098F739927C1
:101D40000895FC01918D828D981731F0828DE80FF6
:101D5000F11D858D90E008958FEF9FEF0895FC01B0
:101D6000918D828D981761F0828DDF01A80FB11DD2
:101D70005D968C91928D9F5F9F73928F90E00895F6
:101D80008FEF9FEF089583E390E1892B49F080E086
:101D900090E0892B29F00E94331081110C940000EF
:101DA0000895FC01848DDF01A80FB11DA35ABF4F18
:101DB0002C91848D90E001968F739927848FA6894A
:101DC000B7892C93A089B1898C9180648C93938D71
:101DD000848D981306C00288F389E02D80818F7D61
:101DE00080830895CF93DF93EC01888D8823C9F019
:101DF000EA89FB89808185FD05C0A889B9898C9114
:101E000086FD0FC00FB607FCF5CF808185FFF2CFAE
:101E1000A889B9898C9185FFEDCFCE010E94D10EA2
:101E2000E7CFDF91CF910895CF92DF92FF920F938A
:101E30001F93CF93DF931F92CDB7DEB76C0181E084
:101E4000D60158968C9358975B969C915B975C96BD
:101E50008C915C97981307C05096ED91FC91519727
:101E6000808185FD2EC0F601038D10E00F5F1F4FAE
:101E70000F731127F02EF601848DF81211C00FB6E2
:101E800007FCF9CFD6015096ED91FC9151978081D6
:101E900085FFF1CFC60169830E94D10E6981EBCF26
:101EA000838DE80FF11DE35AFF4F6083D6015B96E7
:101EB0000C935B975296ED91FC91539780818062D1
:101EC0000CC0D6015696ED91FC91579760835096C1
:101ED000ED91FC91519780818064808381E090E056
:101EE0000F90DF91CF911F910F91FF90DF90CF90D6
:101EF0000895BF92CF92DF92EF92FF92CF93DF933C
:101F0000EC016A017B01B22EE889F98982E08083C5
:101F1000411581EE580761057105A1F060E079E097
:101F20008DE390E0A70196010E94891521503109A7
:101F3000410951095695479537952795211580E117
:101F4000380798F0E889F989108260E874E88EE132
:101F500090E0A70196010E9489152150310941099D
:101F600051095695479537952795EC85FD85308322
:101F7000EE85FF852083188EEC89FD89B082EA8981
:101F8000FB89808180618083EA89FB898081886008
:101F90008083EA89FB89808180688083EA89FB8964
:101FA00080818F7D8083DF91CF91FF90EF90DF90D4
:101FB000CF90BF9008951F920F920FB60F921124E9
:101FC0002F938F939F93EF93FF93E0913605F091BA
:101FD00037058081E0913C05F0913D0582FD12C0FE
:101FE000908180913F058F5F8F732091400582170C
:101FF00051F0E0913F05F0E0EA5DFA4F958F809354
:102000003F0501C08081FF91EF919F918F912F91AA
:102010000F900FBE0F901F9018951F920F920FB642
:102020000F9211242F933F934F935F936F937F935E
:102030008F939F93AF93BF93EF93FF9386E295E0C7
:102040000E94D10EFF91EF91BF91AF919F918F911F
:102050007F916F915F914F913F912F910F900FBEA4
:102060000F901F90189586E295E00E94960E21E051
:10207000892B09F420E0822F0895109229051092EF
:10208000280588EE93E0A0E0B0E080932A059093C5
:102090002B05A0932C05B0932D058EE791E090932E
:1020A00027058093260585EC90E090933305809377
:1020B000320584EC90E0909335058093340580ECF4
:1020C00090E0909337058093360581EC90E09093F3
:1020D00039058093380582EC90E090933B0580931E
:1020E0003A0586EC90E090933D0580933C05109274
:1020F0003F05109240051092410510924205089547
:10210000CF92DF92EF92FF920F931F93CF93DF93C3
:102110007C016A01EB0100E010E00C151D0571F077
:102120006991D701ED91FC910190F081E02DC701FB
:102130000995892B19F00F5F1F4FEFCFC801DF9171
:10214000CF911F910F91FF90EF90DF90CF90089566
:102150006115710581F0DB010D900020E9F7AD01FB
:1021600041505109461B570BDC01ED91FC91028057
:10217000F381E02D099480E090E008950C94A8107C
:10218000DC01ED91FC910190F081E02D09946AE869
:1021900071E00C94A8100F931F93CF93DF93EC0181
:1021A0000E94A8108C01CE010E94C710800F911FC1
:1021B000DF91CF911F910F9108958F929F92AF92CF
:1021C000BF92CF92DF92EF92FF920F931F93CF9324
:1021D000DF93CDB7DEB7A1970FB6F894DEBF0FBE81
:1021E000CDBF7C01C42EE52FCB01D22E19A221E058
:1021F0002D1510F02AE0D22E8E010F5D1F4F8D2C71
:10220000912CA12CB12C6C2D7E2FA50194010E9444
:1022100089158C2DD29E80191124015011098A3004
:1022200014F4805D01C0895CF801808321153105BB
:102230004105510521F0C22EE32FCA01E4CFB801B8
:10224000C7010E94A810A1960FB6F894DEBF0FBE7A
:10225000CDBFDF91CF911F910F91FF90EF90DF9055
:10226000CF90BF90AF909F908F900895CF92DF92C4
:10227000EF92FF920F931F93CF93DF93EC016A01CC
:102280007B012115310579F4E881F9810190F08114
:10229000E02D642FDF91CF911F910F91FF90EF9070
:1022A000DF90CF9009942A303105E9F477FF1AC006
:1022B0006DE20E94C0108C0144275527BA014C19C9
:1022C0005D096E097F092AE0CE010E94DD10800FB2
:1022D000911FDF91CF911F910F91FF90EF90DF90B1
:1022E000CF9008952AE0B701A601CE01DF91CF91EA
:1022F0001F910F91FF90EF90DF90CF900C94DD1025
:102300009A01AB01662757FD6095762F0C94361124
:102310000F931F93CF93DF93EC019A01AB016627D4
:1023200057FD6095762F0E9436118C01CE010E94D8
:10233000C710800F911FDF91CF911F910F910895CA
:102340004F925F926F927F928F929F92AF92BF92C5
:10235000CF92DF92EF92FF920F931F93CF93DF9371
:10236000EC016A017B01B22E9A01AB01C701B601F3
:102370000E946215882319F06DE871E027C02601DC
:102380003701E89477F82FEF3FEF4FE75FE7C3019E
:10239000B2010E94621581110DC02FEF3FEF4FE790
:1023A0005FE7C301B2010E945C1318161CF461E9D7
:1023B00071E00CC02FEF3FEF4FE75FE4C701B601BC
:1023C0000E94B9141816ACF465E971E0CE01DF91F2
:1023D000CF911F910F91FF90EF90DF90CF90BF9022
:1023E000AF909F908F907F906F905F904F900C94E4
:1023F000A8102FEF3FEF4FE75FECC701B6010E9437
:102400005C1387FDE1CF20E030E0A901C701B601F0
:102410000E945C1387FF0AC06DE2CE010E94C010CB
:102420008C01F7FAF094F7F8F09402C000E010E0A5
:10243000A12C60E070E080E09FE3AB1441F020E06D
:1024400030E040E251E40E946013A394F6CF9B0178
:10245000AC01C701B6010E94F8126B017C010E9419
:10246000CD132B013C010E94F9139B01AC01C70164
:10247000B6010E94F7126B017C012AE0B301A201B0
:10248000CE010E94DD10080F191FBB2039F069E949
:1024900071E0CE010E94A810080F191F7B2C772035
:1024A00041F120E030E040E251E4C701B6010E9472
:1024B000BD146B017C010E94C8134B01AA2497FC38
:1024C000A094BA2C2AE030E0B501A401CE010E940C
:1024D0003611080F191FC501B4010E94FB139B019F
:1024E000AC01C701B6010E94F7126B017C017A941E
:1024F000D6CFC801DF91CF911F910F91FF90EF9040
:10250000DF90CF90BF90AF909F908F907F906F9013
:102510005F904F9008950C94A0110F931F93CF9349
:10252000DF93EC010E94A0118C01CE010E94C71024
:10253000800F911FDF91CF911F910F9108954F92BE
:102540005F926F927F92AF92BF92CF92DF92EF92A3
:10255000FF920F931F93CF93DF93CDB7DEB729017F
:102560003A01621B730B840B950B29893A894B89BD
:102570005C892A193B094C095D09298B3A8B4B8BE5
:102580005C8B9B01AC0169897A898B899C890E944B
:102590006D15E418F50806091709A80197010E94AE
:1025A000AB152A0D3B1D4C1D5D1DCA01B901DF9104
:1025B000CF911F910F91FF90EF90DF90CF90BF9040
:1025C000AF907F906F905F904F90089508950E9414
:1025D0003B0D0E94E6120E944706C3ECDEE00E941B
:1025E000B1062097E1F30E94C30EF9CF0895505829
:1025F000BB27AA270ED083C174D130F079D120F047
:1026000031F49F3F11F41EF469C10EF4E095E7FB2D
:1026100051C1E92F85D180F3BA1762077307840788
:10262000950718F071F49EF59DC10EF4E0950B2E00
:10263000BA2FA02D0B01B90190010C01CA01A00114
:102640001124FF27591B99F0593F50F4503E68F16F
:102650001A16F040A22F232F342F4427585FF3CFB0
:10266000469537952795A795F0405395C9F77EF481
:102670001F16BA0B620B730B840BBAF09150A1F0CA
:10268000FF0FBB1F661F771F881FC2F70EC0BA0F50
:10269000621F731F841F48F4879577956795B795D8
:1026A000F7959E3F08F0B3CF9395880F08F09927D0
:1026B000EE0F979587950895D9D008F481E0089595
:1026C0000CD01DC115D140F00CD130F021F45F3F8A
:1026D00019F0F0C0511147C101C122D198F39923DB
:1026E000C9F35523B1F3951B550BBB27AA276217D6
:1026F0007307840738F09F5F5F4F220F331F441F1B
:10270000AA1FA9F333D00E2E3AF0E0E830D0915052
:102710005040E695001CCAF729D0FE2F27D0660F3F
:10272000771F881FBB1F261737074807AB07B0E87E
:1027300009F0BB0B802DBF01FF2793585F4F2AF094
:102740009E3F510568F0B6C00EC15F3FECF3983E66
:10275000DCF3869577956795B795F7959F5FC9F7F1
:10276000880F911D9695879597F90895E1E0660F7A
:10277000771F881FBB1F621773078407BA0720F0F3
:10278000621B730B840BBA0BEE1F88F7E09508955C
:1027900004D06894B111E7C00895CAD088F09F575B
:1027A00090F0B92F9927B751A0F0D1F0660F771F9D
:1027B000881F991F1AF0BA95C9F712C0B13081F07D
:1027C000D1D0B1E00895CEC0672F782F8827B85FA9
:1027D00039F0B93FCCF3869577956795B395D9F7DE
:1027E0003EF490958095709561957F4F8F4F9F4FE8
:1027F0000895E89409C097FB3EF4909580957095F4
:1028000061957F4F8F4F9F4F9923A9F0F92F96E93C
:10281000BB279395F695879577956795B795F111B1
:10282000F8CFFAF4BB0F11F460FF1BC06F5F7F4F4E
:102830008F4F9F4F16C0882311F096E911C0772360
:1028400021F09EE8872F762F05C0662371F096E869
:10285000862F70E060E02AF09A95660F771F881F38
:10286000DAF7880F9695879597F90895990F0008DC
:10287000550FAA0BE0E8FEEF16161706E807F90752
:10288000C0F012161306E407F50798F0621B730BED
:10289000840B950B39F40A2661F0232B242B252B6E
:1028A00021F408950A2609F4A140A6958FEF811D11
:1028B000811D089597F99F6780E870E060E00895B2
:1028C0009F3F31F0915020F4879577956795B795A4
:1028D000880F911D9695879597F908959FEF80EC45
:1028E000089500240A941616170618060906089576
:1028F00000240A9412161306140605060895092EDC
:102900000394000C11F4882352F0BB0F40F4BF2B4A
:1029100011F460FF04C06F5F7F4F8F4F9F4F08958A
:1029200057FD9058440F551F59F05F3F71F0479580
:10293000880F97FB991F61F09F3F79F08795089565
:10294000121613061406551FF2CF4695F1DF08C084
:10295000161617061806991FF1CF869571056105A1
:1029600008940895E894BB2766277727CB0197F949
:1029700008957CDF08F48FEF08950BD0C0CFB1DF4E
:1029800028F0B6DF18F0952309F094CFA7CF1124D3
:10299000EACFC6DFA0F3959FD1F3950F50E0551F06
:1029A000629FF001729FBB27F00DB11D639FAA27A4
:1029B000F00DB11DAA1F649F6627B00DA11D661FF3
:1029C000829F2227B00DA11D621F739FB00DA11D14
:1029D000621F839FA00D611D221F749F3327A00DCE
:1029E000611D231F849F600D211D822F762F6A2F6A
:1029F00011249F5750408AF0E1F088234AF0EE0FEF
:102A0000FF1FBB1F661F771F881F91505040A9F7FB
:102A10009E3F510570F04ECFA6CF5F3FECF3983E3E
:102A2000DCF3869577956795B795F795E7959F5F62
:102A3000C1F7FE2B880F911D9695879597F90895FC
:102A400011F40EF44BCF3CCF73DFD0F39923D9F3BD
:102A5000CEF39F57550B87FF39D00024A0E640EAFC
:102A6000900180585695979528F4805C660F771FE3
:102A7000881F20F026173707480730F4621B730BB6
:102A8000840B202931294A2BA695179407942025D9
:102A900031254A2758F7660F771F881F20F0261721
:102AA0003707480730F4620B730B840B200D311D80
:102AB000411DA09581F7B901842F9158880F9695F3
:102AC00087950895D3DE880B990B08959150504057
:102AD000660F771F881FD2F70895DB018F939F93AE
:102AE0000E94D915BF91AF91A29F800D911DA39F08
:102AF000900DB29F900D11240895991B79E004C0A8
:102B0000991F961708F0961B881F7A95C9F780952C
:102B10000895A1E21A2EAA1BBB1BFD010DC0AA1F1E
:102B2000BB1FEE1FFF1FA217B307E407F50720F036
:102B3000A21BB30BE40BF50B661F771F881F991FB1
:102B40001A9469F760957095809590959B01AC01FA
:102B5000BD01CF010895052E97FB1EF400940E943D
:102B6000C21557FD07D00E94891507FC03D04EF40B
:102B70000C94C21550954095309521953F4F4F4F7D
:102B80005F4F089590958095709561957F4F8F4F19
:102B90009F4F0895A29FB001B39FC001A39F700DE6
:102BA000811D1124911DB29F700D811D1124911D55
:102BB00008950E94CA15A59F900DB49F900DA49FE3
:102BC000800D911D11240895EE0FFF1F0590F491C3
:102BD000E02D0994662777270C94A316FC0188271B
:102BE0009927E89421912032E9F3293010F02E3012
:102BF000C8F32B3241F02D3239F4689404C00E949E
:102C00008516820F911D219120532A30C0F31EF4A6
:102C1000909581959F4F08951F93FC0199278827D0
:102C2000BC01E89411911032E9F3193010F01E3014
:102C3000C8F31B3251F01D3249F4689406C00E945B
:102C40007016610F711D811D911D119110531A3065
:102C5000B0F33EF490958095709561957F4F8F4FBE
:102C60009F4F1F9108959111D1C1803219F0895061
:102C70008550D0F70895FB01DC014150504030F001
:102C80008D910190801919F40020B9F7881B990BD8
:102C90000895FA01A191B081009719F41097E1F01D
:102CA000CD01DC01CD010D90002011F4C00113C055
:102CB000FB012191222319F02015D9F7F3CFFB0155
:102CC0002191201519F41E92119606C02223C1F7F6
:102CD0000D900020A1F7D001FA01A193B0830895CF
:102CE000592F482F372F262F660F771F881F991FC0
:102CF000660F771F881F991F620F731F841F951F10
:102D0000660F771F881F991F08957AE0979F902D6F
:102D1000879F802D910D11240895F999FECF92BDC2
:102D200081BDF89A992780B50895262FF999FECF8D
:102D30001FBA92BD81BD20BD0FB6F894FA9AF99AD8
:102D40000FBE01960895A0E0B0E0E9EAF6E10C9428
:102D500027188B016115710521F0DB018C93119609
:102D60009C93EC015E01BFEFAB1ABB0A7501C880F2
:102D70008C2D90E00E943316892B11F0E501F2CFE3
:102D8000EDE2CE1208C07E01F2E0EF0EF11CC98028
:102D9000DD24D39409C02BE2C21205C07E0142E0BB
:102DA000E40EF11CC980D12CE701219743E050E0EB
:102DB0006AEC70E0CE010E940918892BC1F42396B9
:102DC00045E050E065EC70E0CE010E940918892BC7
:102DD00009F425960115110519F0D801CD93DC935E
:102DE000D11006C160E070E080E89FE70AC143E0CF
:102DF00050E062EC70E0CE010E940918892B59F472
:102E00000115110509F4F9C0B2E0EB0EF11CF8014F
:102E1000F182E082F2C0F70160E070E0CB01C0E037
:102E2000D0E07F01A0EDAA2EAC0C29E02A1530F1EC
:102E30004D2D4260B42E2D2D2870D2FE04C02111DC
:102E400025C0219623C021112197A5E0B0E09B0168
:102E5000AC010E94D915660F771F881F991F6A0D54
:102E6000711D811D911D6839A9E97A078A07A9E1B9
:102E70009A0760F0BD2DB660BB2E08C02EEFA212DF
:102E80000AC0D3FC50C04D2D4860B42E3196D701F6
:102E9000CC90DB2CC6CF2C2D2F7D253409F043C0E0
:102EA000A081AD3241F4BD2DB061DB2E7F0122E067
:102EB000E20EF11C0CC07F01AB3231F04FEFE41A8F
:102EC000F40A21E030E006C0A2E0EA0EF11CA18184
:102ED00022E030E0A053AA3018F0E21AF30A23C02F
:102EE000F70120E030E02038BCE03B075CF4A901AA
:102EF000440F551F440F551F240F351F220F331F3A
:102F00002A0F311DAF014F5F5F4F7A01A081A0539F
:102F1000AA3010F4FA01E7CFD4FE03C03195219511
:102F20003109C20FD31FD1FE09C00115110531F0BF
:102F3000E1E0EE1AF108D801ED92FC920E94F9133B
:102F40002D2D2370233019F04B015C0106C04B017D
:102F50005C01B7FAB094B7F8B09420E030E0A90172
:102F6000C501B4010E945C13882309F43EC0D7FF59
:102F700006C0D195C195D10901EE10E002C009EF5C
:102F800010E06801B8E1CB1AD10890E2E92EF12CEB
:102F9000CE15DF0574F0F8012591359145915491D6
:102FA000C501B4010E94BD144B015C01CE19DF09BB
:102FB000EFCF04501109F594E7940C151D0541F766
:102FC0008A2D880F8B2D881F8F3F49F020E030E03D
:102FD000A901C501B4010E945C13811106C082E2FF
:102FE00090E09093C4058093C305C501B40109C066
:102FF00060E070E080E89FEF04C060E070E080EC8B
:103000009FE7CDB7DEB7ECE00C94431899278827EB
:103010000895FB01DC014150504088F08D918134CE
:103020001CF08B350CF4805E659161341CF06B35BF
:103030000CF4605E861B611171F3990B0895881B77
:10304000FCCF2F923F924F925F926F927F928F921E
:103050009F92AF92BF92CF92DF92EF92FF920F9327
:103060001F93CF93DF93CDB7DEB7CA1BDB0B0FB631
:10307000F894DEBF0FBECDBF09942A8839884888EE
:103080005F846E847D848C849B84AA84B984C88484
:10309000DF80EE80FD800C811B81AA81B981CE0F7B
:1030A000D11D0FB6F894DEBF0FBECDBFED01089560
:1030B00011E0C6E0D1E004C0FE010E94E6152296B0
:0A30C000C830D107C9F7F894FFCF1C
:1030CA000000C505800001000000D007F4010000DF
:1030DA000B0A03090C0D080200001011140F150E3B
:1030EA000607050400000000000000004D313020F2
:1030FA004547472000204100204200205300205528
:10310A0000204400504F532058002059004F4B00D4
:10311A00454747330073657420746F2064656661A0
:10312A00756C742073657475700000000000F60AEF
:10313A00C90A9E0AA60AB90AC80A00000000140FA2
:10314A008010960EAF0EA10EF20E0D0A006E616E81
:0C315A0000696E66006F7666002E0000B3
:00000001FF
